:0E00000012C0FECFFDCFFCCFFBCFFACFF9CF61
:10000E00F8CFF7CFF6CFF5CF24C0F3CFF2CFF1CFA5
:10001E00F0CFEFCFEECFEDCFF894EE27ECBBE5BFF0
:10002E00F8E1A895A4B7A77FA4BFF1BDE1BD8DE00F
:10003E00A2E0ED938A95E9F780E8A0E6ED938A9524
:10004E00E9F7E0E0EAB9EBB9ECB9EFEDEDBFC0E8E6
:10005E0048C264B075B01895E881E7B98BE18A950E
:10006E00F1F7E5B7E77EE862E5BF8895EF7DE5BF7E
:10007E00F30121960895DF98DC98DB98C59AE88104
:10008E00E03029F449D24BD2C298DD9851C0A881F4
:10009E00A13021F4DE9AD998C49847C0A881A23025
:1000AE0039F43AD2C49AC698C298DD9AC39841C020
:1000BE00A881A33031F430D232D2C29ADD9AC398DD
:1000CE0038C0A881A43031F4DE9AD998C498C69A63
:1000DE0029D22FC0A881A53029F4DE98D99A1FD233
:1000EE0021D227C0A881A63039F4DE98D99A17D22A
:1000FE00C298DD98C3981DC0A881A73019F40CD200
:10010E00C49813C0A881A83031F406D208D2C29880
:10011E00DD98C3980EC0A881A93021F4FDD1FFD17E
:10012E0001D207C0DE9AD99AC49AC69AC29ADD9AAB
:10013E00C39AE981E03021F4DF9ADC98DB98C59A06
:10014E00A981A13021F4DF98DC9ADB98C598A981AA
:10015E00A23021F4DF98DC98DB9AC59A88EC90E007
:10016E000197F1F793C15601C0908000D0908100A5
:10017E00E0918200F0918300E0938000F093810083
:10018E00E0918400F0918500E0938200F09383006B
:10019E00E0918600F0918700E0938400F093850053
:1001AE00E0918800F0918900E0938600F09387003B
:1001BE00E0918A00F0918B00E0938800F093890023
:1001CE00E0918C00F0918D00E0938A00F0938B000B
:1001DE00E0918E00F0918F00E0938C00F0938D00F3
:1001EE00E0919000F0919100E0938E00F0938F00DB
:1001FE00E0919200F0919300E0939000F0939100C3
:10020E0095D12ADFE0939200F0939300F601EA0D68
:10021E00FB1DA0918000B09181008BD1A091820036
:10022E00B091830086D1A0918400B091850081D1D8
:10023E00A0918600B09187007CD1A0918800B091EA
:10024E00890077D1A0918A00B0918B0072D1A091D4
:10025E008C00B0918D006DD1A0918E00B0918F0069
:10026E0068D1A0919000B091910063D1A0919200BD
:10027E00B0919300AE0FBF1FE3E2F0E046D24F0104
:10028E00E0EFF0E08E169F0688F4E2E3F0E08E16C3
:10029E009F0660F0F40166277727CAD1ADECBCEC5F
:1002AE008CE89FE3F3D18BD14F0101C04401089537
:1002BE0043D1A438E3E0BE0730F0E9E040D1E45882
:1002CE00F34041D15AC038D1A032E3E0BE0730F03E
:1002DE00E8E035D1E052F34036D14FC02DD1AC3BE2
:1002EE00E2E0BE0730F0E7E02AD1EC5BF2402BD122
:1002FE0044C022D1A835E2E0BE0730F0E6E01FD1BF
:10030E00E855F24020D139C017D1A43FE1E0BE0735
:10031E0030F0E5E014D1E45FF14015D12EC00CD1E0
:10032E00A039E1E0BE0730F0E4E009D1E059F14038
:10033E000AD123C001D1AC32E1E0BE0730F0E3E0D8
:10034E00FED0EC52F140FFD018C0F6D0A83CE0E051
:10035E00BE0730F0E2E0F3D0E85CF040F4D00DC020
:10036E00EBD0A436E0E0BE0730F0E1E0E8D0E45692
:10037E00F040E9D002C0EAE03E2EDED0AA35E0E041
:10038E00BE0730F0E9E0E2D0EA55F040DCD047C0DD
:10039E00D3D0A035E0E0BE0730F0E8E0D7D0E0558E
:1003AE00F040D1D03CC0C8D0A634E0E0BE0730F05B
:1003BE00E7E0CCD0E654F040C6D031C0BDD0DC97DB
:1003CE0028F0E6E0C3D0FC97BED029C0B5D0D297B6
:1003DE0028F0E5E0BBD0F297B6D021C0ADD098970B
:1003EE0028F0E4E0B3D0B897AED019C0A5D05E9790
:1003FE0028F0E3E0ABD07E97A6D011C09DD05497E5
:10040E0028F0E2E0A3D074979ED009C095D01A9739
:10041E0028F0E1E09BD03A9796D001C022248CD0F0
:10042E00199719F4E9E05E2E31C086D0189719F4A9
:10043E00E8E05E2E2BC080D0179719F4E7E05E2E11
:10044E0025C07AD0169719F4E6E05E2E1FC074D040
:10045E00159719F4E5E05E2E19C06ED0149719F4B5
:10046E00E4E05E2E13C068D0139719F4E3E05E2E1D
:10047E000DC062D0129719F4E2E05E2E07C05CD078
:10048E00119719F4E1E05E2E01C0552422960895CD
:10049E00E0E0EBBBEAEFEABBE0E0E8BBECE7E7BB92
:1004AE00E0E0E5BBE3BFE4BBE2BFE3BBE2BBE9BD1B
:1004BE00E0BFEFBDEEBDEDBDECBDEBBDEBBFE5BFEF
:1004CE00E9BFEDB9E0E8E8B9E0E0E9B9E2B9E1B9D0
:1004DE00E2B9E7B9EEE8E6B91F98E3B1E3B978946B
:1004EE000895D6DF40DE36D021D03A92C4DD36D024
:1004FE0031D034D01BD03A92BEDD18D03A92BBDD4B
:10050E0029D02CD04394E9E14E1620F044249A923F
:10051E008A92CEDEE7CFFFCFDE98D9980895C498A1
:10052E00C6980895C29ADD98C3980895E0E0EA93BC
:10053E000895EA0FFB1F0895A881B98108953E2EF4
:10054E00E881F9810895E883F98308952E2EE881D4
:10055E00F9810895E1E0EA932A928DCDE2E0EA93E3
:10056E005A9289CD552342F4503811F4E0FF04C05D
:10057E003196691F791F6BF050E8572711F45F937E
:10058E0073C05F3F31F0660F000C57956795752F5E
:10059E0008955F9300200AF073C06CC050E8192EC6
:1005AE001522880F991F9527550F879550E8072E0E
:1005BE000522660F771F7527550F67950895689466
:1005CE0001C0E8945F93F2DF703818F07F3F08F4B3
:1005DE004BC056E1571BAAF4519558300EF45930C2
:1005EE0030F0EFEFFFEF6FEF7FE777F91AC0772765
:1005FE005523B9F0EE0FFF1F661F771F5A95D1F7DF
:10060E0010C07727583028F0EF2FF62F672F58504D
:10061E00F9CF552331F076956795F795E7955A956D
:10062E00D1F700200AF464D05F910895689401C058
:10063E00E894309760407040B1F0002426F07723A4
:10064E0012F4009455D0172E7EE1112032F07A95D7
:10065E00EE0FFF1F661F111CF9CFEF2FF62F612D26
:10066E005F938ADF5F910895EE27FF27662777272E
:10067E005F910895EFEFFFEF6FE77FEF5F910895C2
:10068E00EFEFFFEF6FE77FE75F9108955F9386DFF0
:10069E00703851F3903841F301240894791F23F4F4
:1006AE001CF300203AF3ECCF3F934F9311243327E2
:1006BE004427552798E1330F441F551FEE1FFF1F88
:1006CE00661F30F43A0F4B1F581FE11DF11D611DBF
:1006DE009A9589F74F913F9166232AF0550FEE1F99
:1006EE00FF1F661F02C07395E3F23CDF5F91089512
:1006FE00F09560957095E195FF4F6F4F7F4F089580
:10070E006F2F660F660B762F08950024112490E14B
:10071E00AA0FBB1F001C111C0E1A1F0A18F40E0E76
:10072E001F1E01C0A1609A9599F7FD01D001089591
:00000001FF
